:10FF1D00E51424FE600E14600F146010240370109D
:10FF2D00F19BC1FD1103C1FD714FC1FDB142C1FD79
:03FF3D00F193221B
:0BFF8100751401F19BF19B917DE1974D
:04FF930075140122BE
:03FEFD00051422C7
:01FF9B002243
:10FF5400C3E5379534FFE5369533FE228510838556
:03FF6400118222E5
:10F80300200E0221DDE51C6416600221DD200C02BE
:10F8130021DD300B0221DDC20ED20BF15460022137
:10F82300DAEF24FE700201BC14700221131470027B
:10F83300216C14700221BC2404600221DAC20BD2B1
:10F843000FE4F532E5227004C2088002D208D1BE6B
:10F85300E524C39410400DE52424F0F50BE434FFB4
:10F86300F50A800CC374109524F50BE49400F50A93
:10F87300C3E50F950BE50E950A5008850E0A850F13
:10F883000B8012E50EC4F854F0C868F50CE50FC4FC
:10F89300540F48F50DE50B450A60024117D3E50FF8
:10F8A3009410E50E940050024117750A00750B1071
:10F8B300E50D150D7002150C22D3E50B9408E50A2E
:10F8C300940040067F08D15C801FAF0BD15C3008E9
:10F8D30007751C0A51438003751C0DE50D450C602B
:10F8E30008E50D150D7002150CE51C640D6008E5A7
:10F8F3001C640A60024117C3E50F9410E50E9400DF
:10F903004007750A00750B1022850E0A850F0B221E
:10F91300D1BEE50FAE0E7803CEC313CE13D8F9F5DF
:10F923000B8E0AE52264017032E4F532F160511D59
:10F93300F51DF4600B85832A85822B7532028016B0
:10F94300E50F150F7002150E0511E5117002051074
:10F95300E50F450E70D3D20FC20B22E5227004C20D
:10F96300088002D208D20FA1FFE52214601F1460A1
:10F973002E146032240360024117E523B4FF077598
:10F983001C067539FF22E4F51C85231E22751C0411
:10F99300E523B4050385243985231F85241D22759A
:10F9A3001C0785241D22E523700775A61E75A6E195
:10F9B3002285258285248341B1E52214600E1460DB
:10F9C300122402704F751C0E85231F22751C05859A
:10F9D300231F22751C0822C20B22300B37E51C643F
:10F9E300167031C20BD20F753201F1547026EF2419
:10F9F300FD601814601714601824037017E50F4591
:10FA03000E6004752A0222E4F52A22A1FFE4F52AF6
:05FA130022851D2A22DE
:10FDFF00E50B450A601B753208E50B150B700215F4
:10FE0F000A74F8250FF50F74FF350EF50ED20B801F
:10FE1F0012E50F450E7002C20F850F32E4F50EF595
:10FE2F000FC20BE4F512E512C39532501FF160308B
:10FE3F000804513B8002511DFF742A2512F8A607B2
:0CFE4F000511E51170020510051280DAA3
:01FE5B002284
:10FEBE00E523F510E524F511E525F508E526F50908
:10FECE00C3E5099511CFE5089510CF2401F50FE490
:04FEDE003FF50E22BC
:02FE5C008F1203
:10FE5E00E4F513E513C39512502FF16074222513A8
:10FE6E00F8E6F51D30080451338002512BE50B15D1
:10FE7E000B7002150A0511E51170020510E50F153C
:09FE8E000F7002150E051380CA65
:01FE97002248
:0EFF6700758FFEE4F521D1E2F181F11D80FCE1
:10FF0000758139E4F521D209D20CD20F752A04A2E9
:0DFF10000C33F52B753202F181F11D80FCE0
:08FFC000B142E51CB416F92260
:10FEE200E5D1B4F0157582015118FFD3947F500A01
:0AFEF200758107E4F5828F8351B19A
:01FEFC0022E3
:10FC7D00E4F583758220511875F010A4F53485F0E4
:10FC8D0033D394F0E53394074005E4F533F534753B
:10FC9D00821F5118F5357582065118F53820092740
:10FCAD0043AB01E538F4601F75821C5118F5B4059E
:10FCBD0082E582700205835118F5B50582E58270E3
:10FCCD000205835118F5B6E4F536F537FFEFC45448
:10FCDD00F0F5B1E4F5B3F5B2F5BCF5BDF5BEF5BF84
:10FCED00F5C4F5C5F5C6F5C70FBF0FE1E4F5B1E5F0
:10FCFD0034AE337803CEC313CE13D8F9F5BC75C427
:10FD0D00FF43B38043B308200920E538F46014E5C0
:10FD1D0038F46016E5B4F4600AE5B5F46005E5B6AF
:10FD2D00B4FF0751C353ABF7D20943AB027582053C
:04FD3D005118F5392B
:01FD4100229F
:10FB4F00E59D600A200907D20951C353ABF7E4F5CD
:10FB5F00B1E5B270028138E5B220E5028138E4F5F3
:10FB6F00B2D209AFBCEF75F008A4FFE5BDC41354C2
:10FB7F0007FDE5F0F536EF4DF537E4F51274222564
:10FB8F0012F8A6A30512E512B408F2C3E5379534AF
:10FB9F00FFE5369533FE60028133EF605D24FE6032
:10FBAF000D14603C14601414603624047076E5392B
:10FBBF00B4FF04D20E806FF140806BE539F460180A
:10FBCF00E523B4050AE524B4FC05E539B4FC09E5E1
:10FBDF00227009E523B4FF04D20E804AF14080461B
:10FBEF00E539B4FC0DB4FC0EE522B40109E523B4EC
:10FBFF000504D20E8030F140802CE522653560057A
:10FC0F00E522F47021E5B3540F64017019100C0450
:10FC1F00D20CC20ED20F752A04A20CE433F52B7549
:10FC2F0032028002C20E43B38075B110E5CF20E1DE
:10FC3F00FBE4F5B2100F0122E536C43354E0FFE5C3
:10FC4F0037131313541F2FF5BCE537C43354E0F5A6
:10FC5F00BDE4F512E512C39532500C742A2512F843
:0DFC6F00E6F5A3051280ED8532B343B340E6
:01FC7C002265
:10FF4000E5342406F537E43533F536D20FE4F52AE7
:04FF500075320122E3
:07FF8C00E4F51D751C1622AF
:04FF9700751C16229D
:10FD4200E51CD198FD6B00FD8603FD9104FD9F0526
:10FD5200FDCA06FDD507FDE008FDED09FD820DFD9A
:10FD6200AD0EFDFE160000FDFB851E83E4F582E567
:10FD72001EC394405004514F80025153751C1622E9
:10FD820051A2E18C851F82851E83511DF51D22E43F
:10FD9200F583851F82E51D5176519AE18CE4F58346
:10FDA200851F825118F51D751C1622E51F14600C63
:10FDB20014600E2402700D751D048008E4F51D8088
:10FDC20003E4F51D751C1622E4F583F5825157757F
:10FDD2001C1622E490000400E51D518EE18CE49093
:10FDE2000004005122F51D751C1622851F82851EF6
:0DFDF20083513BF51D751C1622751C162251
:10FA180075D1FB800875D1F0800375D104E4937526
:10FA2800D1F02275D108F075D1002275D202F07597
:10FA3800D2002275D202E075D2002275D25075D25A
:10FA4800A0E5D220E0FB227840802B7880802774C4
:10FA5800FF900000517675820151767582055176C6
:10FA68007582065176519A7582007800800875D1A2
:10FA78000AF075D1002274FF798012FA2BA3D9FA03
:10FA880012FAA2D8F12275D10CF075D15475D1A40F
:10FA9800800E75D15275D1A2800675D15075D1A04E
:10FAA800E5D120E0FB75D10022E4732275D15075B1
:0BFAB800D1A0E5D120E0FB75D10022B9
:03FFF30002FAB45B
:03F8000002FF758F
:0CFF7500787FE4F6D8FD75813902FF6743
:10FAC300C000C001C002C003780279017A017B0043
:10FAD30043AB0812FB2CE59B20E314200011E5B295
:10FAE30020E5373001F0E59B30E5EBD20080E753AA
:10FAF300ABFDD201C200B8080EBB200280CA0B784E
:10FB03000279017A018008E8B50209B501090812F2
:10FB1300FB2C80CA0A80F80980F575B20075B3889A
:10FB2300D003D002D001D0002275B40075B50075A2
:10FB3300B600EB23F5B4E823F5B5EAC4F5B6E9233B
:0CFB430042B643AB02759B0075B2002275
:10FE9800D083D082F8E4937012740193700DA3A3F9
:10FEA80093F8740193F5828883E47374029368600D
:06FEB800EFA3A3A380DF0D
:00000001FF
